:10000000031E080085015F30A000213084008001BC
:10001000840AA00B07282F2824208400073984068F
:100020000310840C840C840C041A841704128419A1
:10003000841684118A01820701340234043408349E
:10004000103420344034803407398A018207283440
:1000500029342A342B342C342D342E342F340730C9
:10006000B6001930A6207830B600FF30A620033045
:1000700096200530A1200830A12008309A200530B4
:100080009E202B30DA20D7200030C720031D4128C6
:100090006A206A206A206A206A2005309A20083087
:1000A0009E201330B7008830AB2008309A20EA3009
:1000B000B7006030AB2005309E2008309E206430B1
:1000C000AA2005309A2008309A202730B700103037
:1000D000AB205B2805309E206430AA2005309A2092
:1000E0006430AA2005309E206430AA2005309A2072
:1000F0006430AA2005309E206430AA2005309A2062
:100100006430AA2005309E206430AA2005309A2051
:100110006430AA2005309E206430AA2005309A2041
:100120006430AA20E2280730B82093280C208417D6
:100130008004E2280C20FF3A8005A3280C208004CC
:10014000A2280C20FF3A84178005E2288400360894
:100150008000E228B701B600C120640037083604E9
:1001600003190800F730FF3E031DB328C320AD2854
:100170008316F83881050F39810463000F3081043C
:10018000E228B709B609B60A0319B70A0800B90187
:10019000B800CC200239E22839083702031DD428E0
:1001A0003808360203190234031C04340134B70141
:1001B000B600E2280D20BD000005841B3D06031992
:0A01C00000340134831264000800CB
:02400E00DC3F95
:00000001FF
